:100000000C9478040C948A040C948A040C946C2844
:100010000C94D0300C948A040C948A040C948A04B6
:100020000C948A040C948A040C948A040C94C315CE
:100030000C948A040C948A040C948A040C948A0408
:100040000C94DC170C948A040C9457130C94191319
:100050000C948A040C948A040C948A040C948A04E8
:100060000C948A040C948A04F20AAA12AA12FC0ABA
:10007000090B160B230BAA12270BAA12350BAA1277
:100080003F0B490B7A0BAA12AA12AA12530B600B50
:100090006D0B9811A911C811A911CC11DF11D21142
:1000A000D81196219C219F21A221A721AF21B921FE
:1000B000492249224922C121C421CD21D6214922E8
:1000C00049224922492249224922DE21E821F421FC
:1000D000FC21FF2108221122172249224922202235
:1000E000282232223A22132C162C1B2C1E2C212CB7
:1000F000242C272C2A2C2D2C302C332C3F2C3F2C1D
:100100003F2C3F2C3F2C3F2C3F2C3F2C392C362CA6
:100110003C2C862C892C8C2C8F2C922C952C982C5A
:100120009B2C084AD73B3BCE016E84BCBFFDC12F40
:100130003D6C74319ABD56833DDA3D00C77F11BED8
:10014000D9E4BB4C3E916BAAAABE000000803F05DB
:10015000A84CCDB2D44EB93836A9020C50B991860C
:1001600088083CA6AAAA2ABE000000803F003E0DD7
:100170000A002C4C696D3A002C52583A002C4275FA
:10018000663A002C002C57506F733A002C002C4D0F
:10019000506F733A003C446F6F72003C4368656374
:1001A0006B003C416C61726D003C486F6D65003CBA
:1001B000486F6C64003C52756E003C49646C65008D
:1001C0005D0D0A005B302E396A5F70756E63682EB4
:1001D00032303135313032333A000D0A003D0024DF
:1001E0004E005D0D0A00204600205400204D3800CE
:1001F000204D3900204D3500204D3400204D330076
:10020000204D3200204D3100204D30002047393440
:10021000002047393300204739310020473930006A
:10022000204732300020473231002047313900204A
:100230004731380020473137002047004733382EF8
:10024000004738300047330047320047310047301D
:10025000005B005D0D0A005B544C4F3A005D0D0AD7
:10026000002C005B4739323A005D0D0A002C003A41
:10027000003330003238005B47005D0D0A003A0061
:100280002C005B5052423A00290D0A00206D617823
:100290002074726176656C2C206D6D002061636343
:1002A000656C2C206D6D2F7365635E3200206D616F
:1002B0007820726174652C206D6D2F6D696E002C35
:1002C00020737465702F6D6D007A007900780020BE
:1002D00028003D002400202870756E636820736537
:1002E0006E736F7220757020696E766572742C2043
:1002F000626F6F6C290D0A00202870756E6368208C
:1003000073656E736F7220646F776E20696E7665A9
:1003100072742C20626F6F6C290D0A2433333D00F8
:10032000202870756E6368206163747561746F72E4
:1003300020757020696E766572742C20626F6F6C08
:10034000290D0A2433323D00202870756E63682021
:100350006163747561746F7220646F776E20696E6B
:10036000766572742C20626F6F6C290D0A2433310C
:100370003D002028686F6D696E672070756C6C2D6C
:100380006F66662C206D6D290D0A2433303D0020E8
:1003900028686F6D696E67206465626F756E63654E
:1003A0002C206D736563290D0A2432373D00202807
:1003B000686F6D696E67207365656B2C206D6D2F9E
:1003C0006D696E290D0A2432363D002028686F6D54
:1003D000696E6720666565642C206D6D2F6D696E92
:1003E000290D0A2432353D00290D0A2432343D00FE
:1003F0002028686F6D696E672064697220696E7667
:10040000657274206D61736B3A002028686F6D69A6
:100410006E67206379636C652C20626F6F6C290DA9
:100420000A2432333D00202868617264206C696DB3
:100430006974732C20626F6F6C290D0A2432323D6F
:10044000002028736F6674206C696D6974732C20AA
:10045000626F6F6C290D0A2432313D0020287265CD
:10046000706F727420696E636865732C20626F6FA1
:100470006C290D0A2432303D0020286172632074FB
:100480006F6C6572616E63652C206D6D290D0A2499
:1004900031333D0020286A756E6374696F6E206485
:1004A0006576696174696F6E2C206D6D290D0A2463
:1004B00031323D00290D0A2431313D00202873746A
:1004C00061747573207265706F7274206D61736BE7
:1004D0003A00202870726F62652070696E20696E24
:1004E000766572742C20626F6F6C290D0A2431308E
:1004F0003D0020286C696D69742070696E732069F5
:100500006E766572742C20626F6F6C290D0A24362A
:100510003D0020287374657020656E61626C6520F3
:10052000696E766572742C20626F6F6C290D0A24D7
:10053000353D00290D0A24343D00202864697220CD
:10054000706F727420696E76657274206D61736B62
:100550003A00290D0A24333D002028737465702069
:10056000706F727420696E76657274206D61736B42
:100570003A002028737465702069646C6520646596
:100580006C61792C206D736563290D0A24323D005E
:100590002028737465702070756C73652C207573DA
:1005A0006563290D0A24313D0024303D00242420B8
:1005B0002876696577204772626C20736574746968
:1005C0006E6773290D0A2423202876696577202316
:1005D00020706172616D6574657273290D0A24471C
:1005E0002028766965772070617273657220737454
:1005F000617465290D0A244920287669657720628F
:1006000075696C6420696E666F290D0A244E202876
:1006100076696577207374617274757020626C6F8F
:10062000636B73290D0A24783D76616C756520280B
:1006300073617665204772626C2073657474696EAD
:1006400067290D0A244E783D6C696E652028736118
:100650007665207374617274757020626C6F636B61
:10066000290D0A24432028636865636B2067636F44
:100670006465206D6F6465290D0A245820286B6914
:100680006C6C20616C61726D206C6F636B290D0A5C
:100690002448202872756E20686F6D696E6720632C
:1006A00079636C65290D0A7E20286379636C652067
:1006B0007374617274290D0A2120286665656420AF
:1006C000686F6C64290D0A3F202863757272656E2D
:1006D0007420737461747573290D0A6374726C2DC0
:1006E0007820287265736574204772626C290D0A40
:1006F000000D0A4772626C20302E396A5F70756E89
:100700006368205B27242720666F722068656C7001
:100710005D0D0A005D0D0A00526573746F72696E9B
:10072000672064656661756C74730050676D204561
:100730006E6400436865636B20446F6F72004469A8
:100740007361626C656400456E61626C6564004350
:10075000617574696F6E3A20556E6C6F636B65647A
:1007600000272448277C2724582720746F20756E83
:100770006C6F636B00526573657420746F20636FD8
:100780006E74696E7565005B000D0A00486F6D69D7
:100790006E67206661696C0050726F6265206661E9
:1007A000696C0041626F727420647572696E6720B3
:1007B0006379636C6500536F6674206C696D69744E
:1007C0000048617264206C696D697400414C41524B
:1007D0004D3A20000D0A00496E76616C696420670D
:1007E000636F64652049443A00556E646566696EBE
:1007F00065642066656564207261746500556E737A
:100800007570706F7274656420636F6D6D616E6476
:10081000004D6F64616C2067726F75702076696F30
:100820006C6174696F6E004C696E65206F766572DD
:10083000666C6F7700486F6D696E67206E6F74200D
:10084000656E61626C656400416C61726D206C6FF5
:10085000636B004E6F742069646C650045455052AF
:100860004F4D2072656164206661696C2E2055735E
:10087000696E672064656661756C74730056616C9F
:100880007565203C2033207573656300536574746F
:10089000696E672064697361626C65640056616C9F
:1008A0007565203C203000496E76616C6964207368
:1008B000746174656D656E7400426164206E756D5F
:1008C00062657220666F726D617400457870656351
:1008D00074656420636F6D6D616E64206C65747403
:1008E0006572006572726F723A20006F6B0D0A00BC
:1008F00011241FBECFEFD8E0DEBFCDBF26E0A0E0C1
:10090000B1E001C01D92A03DB207E1F70E948C0446
:100910000C94D9370C9400000E94E7120E945522D3
:100920000E945A180E94BF308DE1E7E2F5E0DF0136
:100930001D928A95E9F781E080932705789480914C
:10094000BE0684FF03C081E0809328050E94B51392
:100950000E94AE080E94D6120E941C330E94DA1236
:100960000E941B280E94FB2B0E949B230E942E1892
:100970000E94EB260E94C0081092270510924405A1
:1009800010924605109229050E94E514DFCFEF92E0
:10099000FF921F93CF93DF9300D000D0CDB7DEB787
:1009A0007C01122F8091BE0685FF0BC0C7014983D1
:1009B0005A836B837C830E94342A7C816B815A81A9
:1009C000498180912805823031F149835A836B83B4
:1009D0007C830E94BA138091270581111CC00E945C
:1009E000EA2349815A816B817C81882339F00E94F6
:1009F000DC1449815A816B817C81E7CF212FC701AB
:100A00000F900F900F900F90DF91CF911F91FF905B
:100A1000EF900C94F2230F900F900F900F90DF91B6
:100A2000CF911F91FF90EF9008952F923F924F9298
:100A30005F926F927F928F929F92AF92BF92CF926E
:100A4000DF92EF92FF920F931F93CF93DF93CDB777
:100A5000DEB7E7970FB6F894DEBF0FBECDBF9C8B15
:100A60008B8B1B013A0109871A872B873C87AF8A3A
:100A70002D961FAD2D972E962FAD2E97298B2F9645
:100A80003FAD2F973D8B84E0889EA00111245A83AF
:100A90004983AB89BC89A40FB51FB98FA88F460DB8
:100AA000571D5B8F4A8FFA0180809180A280B380AE
:100AB0002D913D914D915C91C501B4010E94873308
:100AC0006C8F7D8F8E8F9F8FF4E01F9F800111248C
:100AD0002B893C89200F311F39A328A3A301400F84
:100AE000511F5BA34AA3DA014D905D906D907C90FD
:100AF000F9012081318142815381C301B2010E94F9
:100B000087336CA37DA38EA39FA3A50194015058A6
:100B10002D873E874F87588BD301C201B0588D83F4
:100B20009E83AF83B887E981FA81E20DF31D2C8D96
:100B30003D8D4E8D5F8D60817181828193810E9498
:100B400086332B013C01F101E00FF11F2CA13DA1E7
:100B50004EA15FA160817181828193810E94863361
:100B60004B015C01A30192016D857E858F8598897B
:100B70000E949E3669837A838B839C83A5019401AE
:100B80006D817E818F8198850E949E369B01AC018C
:100B900069817A818B819C810E94873369837A8302
:100BA0008B839C83A50194016D857E858F859889B3
:100BB0000E949E364B015C01A30192016D817E81F2
:100BC0008F8198850E949E369B01AC01C501B401BE
:100BD0000E94863329813A814B815C810E94FA33DD
:100BE0002B013C019D89992399F02DEB37E346E0D9
:100BF00055EBC301B2010E94633687FD1DC02BED8A
:100C00003FE049EC50E4C301B2010E94863312C0B8
:100C10002DEB37E346E055E3C301B2010E94603497
:100C2000181654F02BED3FE049EC50E4C301B2013B
:100C30000E9487332B013C018090BA069090BB063E
:100C4000A090BC06B090BD0629853A854B855C8591
:100C5000CA01B9010E948733A50194010E9486331D
:100C60009B01AC01C501B4010E949E360E942B3746
:100C70004B015C0120E030E040E05FE3C301B201E2
:100C80000E949E3629853A854B855C850E949E365A
:100C90009F77A50194010E9467340E943D350E9410
:100CA000D4347E8B6D8BDB01AB2B09F486C14B01F9
:100CB000A12CB12CBF89BB2361F0C501B4010E94F6
:100CC00000359B01AC01C701B6010E949E366B0145
:100CD0007C01C501B4010E9400354B015C019B0100
:100CE000AC01C301B2010E94673469877A878B87A0
:100CF0009C87F989E4E0FE9FC00111242B893C897F
:100D0000280F391F3A8B298BF101E80FF91FD90100
:100D10002D913D914D915C91608171818281938192
:100D20000E948633A50194010E9467346CAB7DABB1
:100D30008EAB9FAB29853A854B855C85CA01B9018D
:100D40000E949E369B01AC0160E070E080E090E480
:100D50000E9486334B015C012BEA3AEA4AE25EE3E9
:100D600069857A858B859C850E949E362B013C0186
:100D700020E030E040E850E4C501B4010E94873330
:100D80009B01AC01C301B2010E949E3668A779A7FE
:100D90008AA79BA720E030E040E05FE3C501B401F3
:100DA0000E949E366CA77DA78EA79FA7198201E09F
:100DB00010E0ED89FE890E171F0709F4FEC0B98106
:100DC000BC3008F04AC02CA53DA54EA55FA56D819D
:100DD0007E818F8198850E949E364B015C0128A5FB
:100DE00039A54AA55BA56D857E858F8598890E946A
:100DF0009E36A50194010E948733B62EA72E982E09
:100E0000892E2CA53DA54EA55FA56D857E858F8578
:100E100098890E949E362B013C0128A539A54AA538
:100E20005BA56D817E818F8198850E949E369B0196
:100E3000AC01C301B2010E9486336D877E878F8724
:100E4000988BE981EF5FE9838B2D9A2DA92DB82D21
:100E50008D839E83AF83B8876EC0B80180E090E039
:100E60000E94003529853A854B855C850E949E3617
:100E70004B015C010E9464346D837E838F8398876D
:100E8000C501B4010E9421374B015C01EA8DFB8D45
:100E900080819181A281B3819C01AD015058298349
:100EA0003A834B835C83AAA1BBA18D919D910D9048
:100EB000BC91A02D88AB99ABAAABBBAB2D813E8179
:100EC0004F81588569817A818B819C810E949E36F1
:100ED0002B013C01A501940168A979A98AA99BA9C4
:100EE0000E949E369B01AC01C301B2010E94873370
:100EF0006D877E878F87988BA501940169817A81A0
:100F00008B819C810E949E364B015C012D813E812C
:100F10004F81588568A979A98AA99BA90E949E3604
:100F20009B01AC01C501B4010E9486336D837E83B1
:100F30008F83988719822D853E854F8558896C8DC2
:100F40007D8D8E8D9F8D0E948733E88DF98D608316
:100F50007183828393832D813E814F8158856CA15B
:100F60007DA18EA19FA10E948733A8A1B9A16D93F5
:100F70007D938D939C9313972CA93DA94EA95FA9AE
:100F8000E989FA8960817181828193810E94873326
:100F9000A989BA896D937D938D939C9313972F891B
:100FA000B701A6018B899C890E94C70480912705FF
:100FB000811121C00F5F1F4FFCCE2F89B701A60101
:100FC000C101E7960FB6F894DEBF0FBECDBFDF912B
:100FD000CF911F910F91FF90EF90DF90CF90BF9036
:100FE000AF909F908F907F906F905F904F903F90C9
:100FF0002F900C94C704E7960FB6F894DEBF0FBE8F
:10100000CDBFDF91CF911F910F91FF90EF90DF90B7
:10101000CF90BF90AF909F908F907F906F905F9098
:101020004F903F902F9008958F929F92AF92BF92D2
:10103000CF92DF92EF92FF924B015C0180912805E5
:10104000823009F447C020E030E040EA51E4C501B5
:10105000B4010E949E360E943D350E94D4346B013B
:101060007C010E94671520E030E04AE754E4C501A6
:10107000B4010E949E364B015C0182E38C9DB0015D
:101080008D9D700D112480E090E00E9400359B0141
:10109000AC01C501B4010E9486330E943D350E9417
:1010A000D434CB010E94DF27C114D10499F00E94EF
:1010B000BA1321E0C21AD1088091270581110AC014
:1010C0008FEF90E722E0815090402040E1F700C090
:1010D0000000EACFFF90EF90DF90CF90BF90AF90ED
:1010E0009F908F9008950E94102881E00E94A02870
:1010F0000E94BA1380912705811104C00E94C00884
:101100000C941B2808958091440584FD26C09FB748
:10111000F894809144058061809344059FBF0E94AC
:10112000D7120E94DB1280912805982F9C7021F421
:1011300090912905913089F49FB7843029F4F8946F
:1011400080914605806204C0F894809146058860CD
:10115000809346059FBF0C949815089580E4E7E4BA
:10116000F5E0DF011D928A95E9F76BE675E080E016
:101170000E94F620811103C087E00C94FD2B089596
:101180006AE275E08FE595E00C94BC322F923F92B5
:101190004F925F926F927F928F929F92AF92BF9287
:1011A000CF92DF92EF92FF920F931F93CF93DF9333
:1011B000CDB7DEB7AB970FB6F894DEBF0FBECDBF8D
:1011C00098A38F8F8AE3E7E8F5E0DF011D928A9507
:1011D000E9F78BE0E7E4F5E0A8E8B5E001900D92CF
:1011E0008A95E1F71D8E212C312CA12CB12C19A24E
:1011F000512C1E8E66246394712C58E0452E992440
:10120000939465E0862E8D8DEF8DF8A1E80FF11D8A
:101210000081002309F491C29FEB900F9A3110F0E6
:101220000C949C128F5F8D8FAE01475E5F4FBE01A5
:10123000635E7F4F8F8D98A10E942D27882311F424
:101240000C949E12C98CDA8CEB8CFC8CC701B60115
:101250000E946C370E94D434162F70E080E090E03A
:101260000E9402359B01AC01C701B6010E94863382
:1012700020E030E048EC52E40E949E360E940137A4
:101280000E94D434073421F00D3409F450C199C1BF
:10129000183209F432C1E8F4143160F4113108F065
:1012A000D7C0143009F45AC008F48EC01A30D9F1EE
:1012B0000C94AA121C31B9F128F4163108F4F7C0C5
:1012C0000C94AA121E3179F1163209F47DC00C94E7
:1012D000AA121D3309F40BC1A8F4153309F461C037
:1012E00040F41B3209F4ECC0113309F4E9C00C944A
:1012F000AA121C3310F00C94AA12165310938E05E8
:1013000089E000C11C3540F41A3508F0B0C0103532
:1013100009F49BC00C94AA121C3529F01F3508F45F
:10132000BDC00C94AA126115710531F4BE8DB111C6
:101330000C94A012E1E0EE8F1C3199F038F41430D7
:1013400069F01A3009F0DBC082E02CC0153349F196
:101350001C3559F11E3109F0D2C013C09092870597
:10136000CEC06115710549F06A30710511F00C9419
:10137000AA1224E02093870509C0F3E0F0938705C3
:1013800005C06115710521F48092870580E0BFC01A
:101390006A30710511F00C94AA1236E0309387057B
:1013A000F5CF87E080938705AAC06115710549F0E4
:1013B0006A30710511F00C94AA1299E09093870598
:1013C000E5CF40928705E2CFAE8DA1110C94A0121B
:1013D000B2E0BE8F123089F028F4112359F0113099
:1013E00081F08FC0163281F0103579F1133009F099
:1013F00088C007C01092880584C0EE8DE0938805F0
:1014000080C0109388057DC06E317105B1F048F43D
:101410006431710511F00C94AA12F4E0F093880580
:1014200012C06832710561F06233710511F00C94DD
:10143000AA1237E03093880506C08092880503C061
:1014400026E02093880581E062C04092880559C05B
:10145000123129F0133139F010928C0502C09092AC
:101460008C0582E04FC082E080938C054BC06115F3
:10147000710549F41A3519F410928B0502C0909247
:101480008B0583E044C06A30710511F00C94AA12F8
:101490001A3511F40C94AA1284E039C01D3519F4E0
:1014A0009092890502C01092890585E02BC0143105
:1014B00019F490928A0502C010928A0586E022C033
:1014C0008E8D81110C94A012113331F410928D0580
:1014D00088E093E09E8F1BC06A30710511F00C9478
:1014E000AA1290928D0588E0A3E0AE8F10C0672B02
:1014F00011F00C94AA128AE00AC087E003C080E0D1
:1015000001C081E0672B19F087E10C94BD12F30153
:1015100002C0EE0FFF1F8A95E2F7CF019F012A213B
:101520003B21232B09F44AC085E10C94BD12672BA3
:1015300059F7163018F4133090F01EC01E31C1F068
:1015400030F488EF810F823030F10C94AA121436F7
:1015500011F00C94AA12909292058EE027C01230DE
:1015600039F01E3129F0111120C090928F051DC055
:1015700082E080938F0519C0143029F0153039F0BE
:101580009092910506C082E08093910502C010926E
:1015900091058CE00BC0193021F082E0809390051A
:1015A00002C0109290058DE001C08BE0930102C053
:1015B000220F331F8A95E2F7C901B1CFA82AB92AB1
:1015C00022CE802F992787FD9095A92FB92FFC0156
:1015D000E654F109E531F10508F0BCC7EC5CFF4FBA
:1015E0000C94B937C0929305D0929405E09295057A
:1015F000F092960580E07FC0C0929705D092980542
:10160000E0929905F0929A0539A1316039A381E001
:1016100072C0C0929B05D0929C05E0929D05F0920D
:101620009E0589A1826089A382E065C0C0929F0562
:10163000D092A005E092A105F092A20599A1946034
:1016400099A383E058C01093A30584E054C0C70158
:10165000B6010E94CF346093A4057093A5058093D2
:10166000A6059093A70585E046C0C092A805D09234
:10167000A905E092AA05F092AB0586E03CC0C092B5
:10168000AC05D092AD05E092AE05F092AF0587E0D3
:1016900032C0C092B005D092B105E092B205F0928E
:1016A000B30588E028C0C092B505D092B605E09297
:1016B000B705F092B805A52DA1605A2E8AE01BC08F
:1016C000C092B905D092BA05E092BB05F092BC0574
:1016D000B52DB2605B2E8BE00EC0C092BD05D092DE
:1016E000BE05E092BF05F092C005E52DE4605E2ED8
:1016F0008CE001C089E08301082E02C0000F111F99
:101700000A94E2F7980122213321232B09F01AC70A
:1017100021E633E002C0359527958A95E2F720FF50
:1017200009C020E030E0A901C701B6010E94603481
:1017300087FD0AC7202A312A66CD552029F03E8D23
:10174000311102C082E08E8F25FE0EC08091A4056B
:101750009091A505A091A605B091A705803896495E
:10176000A849B1050CF0F2C680918905813031F4A9
:10177000FE8DF230A1F520FEF3C631C08091480500
:1017800081112DC020FE1BC080918A05813039F562
:1017900023E333E34BEC51E460919305709194059E
:1017A00080919505909196050E949E3660939305D1
:1017B00070939405809395059093960510C0809141
:1017C000560590915705A0915805B0915905809301
:1017D000930590939405A0939505B093960530FCDE
:1017E00010C08091520590915305A0915405B0917D
:1017F00055058093B0059093B105A093B205B093C1
:10180000B30580918705813031F426FC02C08CE15C
:10181000B4C6E89426F880918C05882341F0813085
:1018200061F019A682E088A791E09FA30BC022E097
:1018300029A731E038A71FA205C0A1E0A9A718A6D3
:10184000B2E0BFA380918A05813021F0EE8DE330B4
:1018500091F52AC035EBE32E35E0F32E00E010E0E1
:10186000C52CD12CC601002E02C0959587950A94EF
:10187000E2F780FF10C023E333E34BEC51E4D701E0
:101880006D917D918D919C910E949E36F7016083B0
:101890007183828393830F5F1F4FF4E0EF0EF11C7F
:1018A00003301105F9F6D2CF80918D05813019F4FE
:1018B00024E052124DC68CE0EBE6F5E0DE011D9609
:1018C00001900D928A95E1F7B1FC09C0309187052E
:1018D0003F8F3230B9F0383009F4B0C015C1809173
:1018E0008E05873010F08DE148C690914D05981710
:1018F00069F3BE01635F7F4F0E94F620882309F4DD
:1019000039C6E4CF511002C08AE137C6C1018075E3
:101910009927892B09F47BCF6091A8057091A905BF
:101920008091AA059091AB050E946C370E94D43437
:101930006730C8F68091A305843129F0823009F020
:1019400009C627FC07C68FEA2822662319F06150D2
:101950006F8F03C090918E059F8FBE016F5F7F4F89
:101960008F8D0E94F620882309F404C64090A305B9
:101970006090830570908405809085059090860521
:10198000DE0111967D0195EBC92E95E0D92E2FE54C
:10199000A22E25E0B22E00E010E0E52DF0E0FEA33F
:1019A000EDA38DA19EA1002E02C0959587950A9466
:1019B000E2F780FF33C0F4E14F1226C0D5015896FC
:1019C0002D913D914D915C915B976D917D918D91A4
:1019D0009C910E948633F60120813181428153819E
:1019E0000E948633D7016D937D938D939C931397BB
:1019F0000230A1F4A40193010E948633F7016083B1
:101A00007183828393830AC0F60180819181A281D0
:101A1000B381F70180839183A283B3830F5F1F4F4C
:101A2000F4E0EF0EF11C24E0C20ED11C34E0A30E52
:101A3000B11C0330110509F0B4CF0FC1552009F4D2
:101A400063CF6090830570908405809085059090A9
:101A5000860505EB15E08FE5C82E85E0D82E5E01E2
:101A60008DE0A80EB11CE12CF12CA52DB0E0B8A39F
:101A7000AF8F8F8D98A10E2C02C0959587950A94F3
:101A8000E2F780FF26C0F501208131814281538138
:101A9000D6016D917D918D919C910E948633F801C4
:101AA00020813181428153810E948633D8016D9318
:101AB0007D938D939C931397B2E0EB1214C0A40115
:101AC00093010E948633F80160837183828393833C
:101AD0000AC0F601808D918DA28DB38DF8018083AF
:101AE0009183A283B383FFEFEF1AFF0A0C5F1F4FAE
:101AF00024E0C20ED11C34E0A30EB11C83E0E81632
:101B0000F10409F0B6CFA8C09E8D933059F4AF8D83
:101B1000A53009F48FC0A73009F499C0A33009F0AB
:101B20009BC080C0552099F340908B058090830521
:101B300090908405A0908505B09086050FE5C02E95
:101B400005E0D02E05EB15E03E01BDE06B0E711CEB
:101B5000E12CF12CE52DF0E0FEA3EDA38DA19EA1DB
:101B60000E2C02C0959587950A94E2F780FD0BC074
:101B7000F60180819181A281B381F80180839183F4
:101B8000A283B3833EC0FF8DF730D9F1411028C046
:101B9000D60158962D913D914D915C915B97F30143
:101BA00060817181828193810E948733D8012D9158
:101BB0003D914D915C910E948733F8016083718360
:101BC00082839383F2E0EF121CC0A50194010E946E
:101BD0008733D8016D937D938D939C93139711C098
:101BE000F6012081318142815381D8016D917D912F
:101BF0008D919C910E948733F80160837183828369
:101C00009383FFEFEF1AFF0A24E0C20ED11C0C5F92
:101C10001F4F34E0630E711C83E0E816F10409F0F5
:101C20009DCF75CF511001C01E8EBE016F5F7F4FDB
:101C300086E007C0511001C01E8EBE016F5F7F4F4E
:101C400087E00E94F620882309F494C405C080919F
:101C50008805823008F080C41F8E109188051830E6
:101C600041F4552009F4B2C19E8D913009F076C43B
:101C700089C2AE8DA23009F0A9C11123D9F020E0AC
:101C800030E0A901609193057091940580919505CC
:101C9000909196050E946034882309F461C4143041
:101CA00028F4123058F4113029F06CC2183008F4BE
:101CB0004CC168C2511066C21E8E8BC1552009F4FA
:101CC00023CEFFA1EF2FF0E0FEA3EDA338A5232F35
:101CD00030E03BA72AA781E090E03C0108A402C0C5
:101CE000660C771C0A94E2F70FA002C0880F991FB8
:101CF0000A94E2F7682A792A852D90E086219721B7
:101D0000892B09F42FC4EE0FFF1FEE0FFF1FE957B9
:101D1000FA4FADA1BEA1AA0FBB1FAA0FBB1FA15AAC
:101D2000BA4F2D913D914D915C9166A577A580A903
:101D300091A90E9486336B017C01EAA5FBA5EE0FF9
:101D4000FF1FEE0FFF1FE957FA4FAAA5BBA5AA0F69
:101D5000BB1FAA0FBB1FA15ABA4F2D913D914D91A8
:101D60005C9166A577A580A991A90E9486334B0155
:101D70005C0127FE40C0E89427F82091B50530911A
:101D8000B6054091B7055091B80560915F05709117
:101D9000600580916105909162050E946034811117
:101DA0001CC12091B9053091BA054091BB055091F5
:101DB000BC05609163057091640580916505909103
:101DC00066050E946034811108C12091BD053091E3
:101DD000BE054091BF055091C005609167057091A7
:101DE00068058091690590916A050E9460348111AF
:101DF000F4C081E2C2C3F9A14F2E512C642075209A
:101E0000672809F4B1C321EF222280918A0581302D
:101E100009F456C00AA51BA5000F111F000F111FC2
:101E200009561A4FD8012D913D914D915C91C501F4
:101E3000B4010E9486332B013C01ADA0BEA0AA0CC8
:101E4000BB1CAA0CBB1CF501E956FA4F5F012081AF
:101E5000318142815381C701B6010E948633A301BB
:101E600092010E94EA276B017C01D8012D913D91DE
:101E70004D915C91F50160817181828193810E9415
:101E8000EA274B015C016093AC057093AD0580932C
:101E9000AE059093AF059B01AC01C701B6010E944E
:101EA00086336B017C01E894F7F82AE037ED43EACA
:101EB0005BE3C701B6010E94633618164CF162C19C
:101EC00087E9682E85E0782E00E010E0C201002E40
:101ED00002C0959587950A94E2F780FF10C023E32E
:101EE00033E34BEC51E4D3016D917D918D919C9145
:101EF0000E949E36F30160837183828393830F5F18
:101F00001F4FF4E06F0E711C03301105F9F682CFFC
:101F100020E030E040E05FE3C701B6010E94633695
:101F200018160CF466CF2FE632E143E85AE3C501F8
:101F3000B4010E949E369B01AC01C701B6010E940C
:101F4000633618160CF455CF1DC1552009F4DCCCAE
:101F50002091B5053091B6054091B7055091B8056F
:101F600060915F05709160058091610590916205B7
:101F70000E946034811106C12091B9053091BA05E3
:101F80004091BB055091BC0560916305709164055B
:101F900080916505909166050E9460348111F2C0C0
:101FA0002091BD053091BE054091BF055091C005FF
:101FB00060916705709168058091690590916A0547
:101FC0000E946034882309F414CFDCC02E8D2111C7
:101FD000D9C0C1018E7D9C7FD8C080918A05813097
:101FE000B1F423E333E34BEC51E46091AC05709121
:101FF000AD058091AE059091AF050E949E3660932D
:10200000AC057093AD058093AE059093AF054090FD
:10201000AC055090AD056090AE057090AF0520E026
:1020200030E040E850E4C301B2010E949E36A301B3
:1020300092010E949E362B013C01A7019601C70127
:10204000B6010E949E369B01AC01C301B2010E9401
:1020500086332B013C01A5019401C501B4010E9406
:102060009E369B01AC01C301B2010E9486332B0155
:102070003C0120E030E0A9010E94603487FD7CC271
:10208000C301B2010E942B372B013C01A501940131
:10209000C701B6010E94EA279B01AC01C301B2014E
:1020A00090580E9467342B013C0180918805833051
:1020B00021F477FA709477F870948091AC05909140
:1020C000AD05A091AE05B091AF0589A39AA3ABA3CE
:1020D000BCA320E030E0A901BC01CD010E94603426
:1020E00087FF11C077FA709477F8709489A19AA14C
:1020F000ABA1BCA1B0588093AC059093AD05A09363
:10210000AE05B093AF050DA11EA1000F111F000F6A
:10211000111F09561A4FA3019201C501B4010E9473
:102120009E369B01AC01C701B6010E94863320E0B8
:1021300030E040E05FE30E949E36D8016D937D93CE
:102140008D939C9313970AA51BA5000F111F000FD9
:10215000111F09561A4FA3019201C701B6010E942F
:102160009E369B01AC01C501B4010E94873320E07B
:1021700030E040E05FE30E949E36F80160837183A7
:1021800082839383C1018E7D907E892B09F0EEC1FD
:102190008091A4059091A505A091A605B091A705F1
:1021A00080935B0590935C05A0935D05B0935E05FD
:1021B00080918905809348058091930590919405BD
:1021C000A0919505B091960580935605909357057B
:1021D000A0935805B0935905C090B005D090B105B3
:1021E000E090B205F090B305A70196016091520509
:1021F0007091530580915405909155050E9460346B
:102200008823C1F080915005882321F0B701A601F1
:102210000E94D9128091B0059091B105A091B205AC
:10222000B091B3058093520590935305A093540544
:10223000B09355058091B40580935A05809191051E
:1022400090915005981771F04091520550915305A7
:1022500060915405709155050E94D91280919105A5
:10226000809350058091900590914F05981731F01B
:102270000E94DD128091900580934F058091870523
:10228000813051F46091A8057091A9058091AA054B
:102290009091AB050E94140880918C0580934B05AA
:1022A00080918A05809349053E8D3330F9F4809101
:1022B0008D0580934C05813089F48091BD05909106
:1022C000BE05A091BF05B091C00580938305909392
:1022D0008405A0938505B093860508C010928305F8
:1022E00010928405109285051092860580918E05C6
:1022F00090914D05981759F080934D058CE0FE01A3
:102300003D96ABE6B5E001900D928A95E1F780919C
:102310008B0580934A058091870590E0FC013297F8
:10232000E830F10508F04BC0E75BFF4F0C94B9377C
:10233000BE016F5F7F4F8F8D0E94A61F80914D055C
:102340009F8D89133CC08CE0FE013196ABE6B5E071
:102350001AC0AE8DAA2349F020E040E050E060E8CA
:102360007FEB85EB95E00E94C70420E040E050E061
:1023700060E87FEBCE0101960E94C7048CE0FE016D
:102380003196AFE5B5E001900D928A95E1F717C05F
:102390006FE575E086E003C06FE575E087E00E94B9
:1023A000A61F0DC08CE0E5EBF5E0A7E7B5E0EBCFAD
:1023B0008CE0E7E7F5E0DF011D928A95E9F780916F
:1023C000880580934705883009F464C0BE8DB2301B
:1023D00009F060C0813011F1D8F0823071F18330A2
:1023E00009F04FC0C0905605D0905705E0905805B1
:1023F000F09059050091AC051091AD052091AE0506
:102400003091AF051F9289A58F9398A59F932BC0FC
:1024100020E040E050E060E87FEB0AC040915605C4
:1024200050915705609158057091590520914805C4
:1024300085EB95E00E94C70424C0C0905605D0905B
:102440005705E0905805F09059050091AC051091A2
:10245000AD052091AE053091AF0581E08F93E9A5E0
:10246000EF93F8A5FF938FA0A090480547E955E0AA
:1024700065EB75E08FE595E00E9415050F900F90D4
:102480000F908CE0E5EBF5E0AFE5B5E001900D9243
:102490008A95E1F78091920580935105813021F46E
:1024A0000E945D331092510580918F0580934E05F7
:1024B000882309F45DC00E94671590914E058091B4
:1024C0002805913069F48230A1F19FB7F89480918A
:1024D00044058860809344059FBF0E94BA1329C0B9
:1024E00091E09093470510924B0510924A05109287
:1024F000480510924D051092500510924F058230FC
:10250000A9F0BE01635F7F4F80E00E94F620882320
:1025100089F18CE0FE013D96ABE6B5E001900D92AD
:102520008A95E1F70E94D7120E94DB1287E00E9491
:10253000752C10924E051CC081E01FC082E01DC0AA
:1025400088E11BC089E119C084E017C08BE115C088
:1025500085E213C084E111C08EE10FC08FE10DC090
:1025600086E10BC080E209C083E207C084E205C0B7
:1025700080E003C087E001C082E2AB960FB6F8941A
:10258000DEBF0FBECDBFDF91CF911F910F91FF90A6
:10259000EF90DF90CF90BF90AF909F908F907F9003
:1025A0006F905F904F903F902F90089508950895F9
:1025B0000895089508950895089508959091020149
:1025C00080910301891708F48058891B0895E0EC75
:1025D000F0E08081826080831092C50080E180936A
:1025E000C400E1ECF0E080818061808380818860BC
:1025F00080838081806880830895E091010191E06B
:102600009E0F903409F490E020910001921305C0D0
:102610002091440524FFF8CF0895F0E0EF53FA4FDE
:102620008083909301018091C10080628093C100FA
:1026300008951F920F920FB60F9211248F939F93BC
:10264000EF93FF9380910001E82FF0E0EF53FA4FF2
:1026500090819093C6008F5F803409F480E080936E
:10266000000190910101891305C08091C1008F7D07
:102670008093C100FF91EF919F918F910F900FBEBA
:102680000F901F9018959091020180910301891776
:1026900061F0E92FF0E0EF5FF94F80819F5F9038A4
:1026A00009F490E09093020108958FEF08951F922E
:1026B0000F920FB60F9211242F933F934F935F9376
:1026C0006F937F938F939F93AF93BF93EF93FF93FA
:1026D0008091C6008F33A9F050F4883109F181321E
:1026E00011F59FB7F89480914405886015C0803437
:1026F00071F08E37C1F49FB7F894809144058260E1
:102700000BC09FB7F89480914405816005C09FB7C6
:10271000F894809144058062809344059FBF14C063
:102720000E94830811C0E091030191E09E0F903850
:1027300009F490E020910201921731F0F0E0EF5F90
:10274000F94F808390930301FF91EF91BF91AF9177
:102750009F918F917F916F915F914F913F912F91B9
:102760000F900FBE0F901F901895809103018093DA
:1027700002010895EF92FF920F931F93CF93DF937F
:10278000D1E008E080E2F82E10E190E4E92EC0915B
:102790004605CC2389F1D0932805C1FF02C081E012
:1027A0000FC0C2FF02C082E00BC0C3FF02C083E0C3
:1027B00007C0C4FF02C084E003C0C5FF03C085E0BA
:1027C0000E944B2CC0FD08C08FB7F894909146052D
:1027D000109246058FBF10C081E00E94752C9FB7F4
:1027E000F894809144058F7E809344059FBF80912B
:1027F000440584FFFCCFE8CFC0914405CC2309F405
:10280000BCC0C4FF04C081E080932705CEC0C0FFD8
:102810000AC00E94C02F9FB7F894809144058E7F14
:10282000809344059FBF8C2F887609F43CC080912B
:102830002805882349F0982F9C7769F1883021F486
:102840000E947C18D093290580912805811103C02E
:1028500092E090932905C6FF09C0883011F4E092F8
:10286000280580912905886080932905C3FF05C04C
:102870008091280585FF10932805C5FF0CC086E0D0
:102880000E94752C8091290581FDC460846080932D
:102890002905F09228059FB7F8948091440587791F
:1028A000809344059FBFC1FF48C08C2F8876E9F50F
:1028B00080912805882331F08075B9F18091290530
:1028C00081FF33C08091290582FF1CC08091500593
:1028D000882371F040915205509153056091540541
:1028E000709155050E94D81280EA9FE00E94DF2770
:1028F00080914F05882331F00E94DC1288EE93E02E
:102900000E94DF270E94C023892B59F0809129055E
:1029100083FD07C0009328050E949E180E94781529
:1029200002C010922805109229059FB7F894809153
:1029300044058D7F809344059FBFC2FF1EC08091D8
:102940002805807371F08091290582FF04C00E94E0
:10295000D7120E94DB12809129058260809329059D
:1029600004C010922905109228059FB7F894809111
:1029700044058B7F809344059FBF809128058C7709
:1029800011F00E949E1880912805803251F48091A8
:10299000290581FF06C00E940931811102C01093F0
:1029A0002805809129058111F2CEDF91CF911F91E9
:1029B0000F91FF90EF9008959FB7F8948091440590
:1029C0008260809344059FBF0895CF93DF930E9458
:1029D000A42C80912805813021F482E00E94752C7E
:1029E0002FC00E940931882341F080914405806204
:1029F000809344050E94BA1302C01092280584E017
:102A000091E00E940B311CC08D3079F0DD2399F1EB
:102A1000893221F4D13009F04CC0D0E00E94431338
:102A20008F3F09F448C08A3079F7EC2FF0E0EC5F73
:102A3000FE4F10820E94BA1380912705882311F05F
:102A4000C0E0EBCF80910401811103C00E94FD2BF7
:102A5000F7CF843229F484E091E00E942A31F6CF46
:102A600080912805813011F489E0F0CF84E091E075
:102A70000E94C608EBCF813288F28F3279F2883219
:102A8000B1F08B33B1F0CF3428F08BE00E94FD2BF6
:102A9000C0E0C4CF2C2F30E0CF5F9FE9980FF90141
:102AA000EC5FFE4F9A3108F480528083B7CFD1E0BB
:102AB000B5CFD2E0B3CF0E94DC140E94BA1380914C
:102AC0002705882309F4AACFDF91CF9108950E94AA
:102AD000DC140E94BA1380912705811108C00E945E
:102AE000C023892BB1F780912805883091F3089590
:102AF0008091BE0682FF02C0289A01C0289880916A
:102B000028058C70A1F080918401809398018091B8
:102B10008501809397018091B106880F845081953B
:102B20008093960180916F00826080936F0008957A
:102B300080916F008D7F80936F0080918100887FEE
:102B4000816080938100109283018091B4068F3F51
:102B500021F490914605992349F0909128059430ED
:102B600029F090E00E94DF2781E001C080E0909191
:102B7000BE0692FF02C091E08927882311F0289AAF
:102B80000895289808951F920F920FB60F9211245E
:102B90002F933F934F935F936F937F938F939F9365
:102BA000AF93BF93CF93DF93EF93FF938091830114
:102BB0008111EFC19BB180919801807E9F71892B1B
:102BC0008BB98BB1837E90919701892B8BB98091C2
:102BD000960186BD82E085BD81E080938301789473
:102BE0008091AA019091AB01892B09F0A4C080913A
:102BF000880190918701981709F492C0E0918801AB
:102C000086E0E89FF0011124E455FE4FF093AB01FC
:102C1000E093AA0183819481909389008093880036
:102C2000808191819093A6018093A501A2818091DA
:102C3000A7018A1771F1A093A70181E1A89FD00194
:102C40001124A053BE4FB093A901A093A8011D96D3
:102C50008D919D910D90BC91A02DB695A7959795BE
:102C600087958093910190939201A0939301B093E3
:102C7000940180938D0190938E01A0938F01B09366
:102C800090018093890190938A01A0938B01B09366
:102C90008C01C091A801D091A901809184019881F3
:102CA000892780939801258189819A81AB81BC8194
:102CB000022E04C0B695A795979587950A94D2F7EA
:102CC0008093990190939A01A0939B01B0939C01EA
:102CD0008D819E81AF81B885022E04C0B695A795DF
:102CE000979587950A94D2F780939D0190939E01C2
:102CF000A0939F01B093A00189859A85AB85BC857F
:102D000004C0B695A795979587952A95D2F7809395
:102D1000A1019093A201A093A301B093A4010BC0C1
:102D20000E9498159FB7F894809144058460809321
:102D300044059FBF2EC10E94FC2B109297018091E9
:102D4000990190919A01A0919B01B0919C014091B1
:102D5000890150918A0160918B0170918C01840FDF
:102D6000951FA61FB71F8093890190938A01A09396
:102D70008B01B0938C01E091A801F091A9014585E8
:102D8000568567857089481759076A077B0768F574
:102D900024E0209397014585568567857089841BBB
:102DA000950BA60BB70B8093890190938A01A09392
:102DB0008B01B0938C01208180912A0590912B0585
:102DC000A0912C05B0912D0525FF04C00197A10904
:102DD000B10903C00196A11DB11D80932A059093EE
:102DE0002B05A0932C05B0932D0580919D0190910A
:102DF0009E01A0919F01B091A00140918D01509141
:102E00008E0160918F0170919001840F951FA61F14
:102E1000B71F80938D0190938E01A0938F01B09383
:102E200090014585568567857089481759076A0757
:102E30007B0778F5209197012860209397014585BD
:102E4000568567857089841B950BA60BB70B8093FD
:102E50008D0190938E01A0938F01B09390012081FA
:102E600080912E0590912F05A0913005B0913105EC
:102E700026FF04C00197A109B10903C00196A11D55
:102E8000B11D80932E0590932F05A0933005B0932C
:102E900031058091A1019091A201A091A301B0916F
:102EA000A401409191015091920160919301709120
:102EB0009401840F951FA61FB71F809391019093D3
:102EC0009201A0939301B09394014585568567853F
:102ED0007089481759076A077B0778F52091970191
:102EE0002061209397014585568567857089841BED
:102EF000950BA60BB70B8093910190939201A09331
:102F00009301B09394012081809132059091330513
:102F1000A0913405B091350527FF04C00197A109A0
:102F2000B10903C00196A11DB11D80933205909394
:102F30003305A0933405B09335058091280584307E
:102F400039F48091430590919701892380939701EB
:102F50008091A5019091A60101979093A60180937D
:102F6000A501892B69F41092AB011092AA018091FE
:102F700088018F5F80938801863011F41092880158
:102F800080918501909197018927809397011092F4
:102F90008301FF91EF91DF91CF91BF91AF919F910D
:102FA0008F917F916F915F914F913F912F910F90F2
:102FB0000FBE0F901F9018951F920F920FB60F9291
:102FC00011248F939F939BB1809185018C71937E87
:102FD000892B8BB915BC9F918F910F900FBE0F90CD
:102FE0001F901895FF920F931F93CF93DF9310922A
:102FF000850110928401C0E0D0E00C2F1C2F20919D
:10300000B20630E08C2F0C2E02C0359527950A941D
:10301000E2F720FF07C0F09085010E9462228F290D
:10302000809385012091B30630E002C03595279545
:103030001A95E2F720FF08C010918401802F0E94AA
:103040006C22812B809384012196C330D105A9F68F
:10305000DF91CF911F910F91FF9008950E949815D5
:103060008BE2E4E5F1E0DF011D928A95E9F783E266
:10307000E9E8F1E0DF011D928A95E9F710928201FB
:1030800010928101109288011092870181E0809353
:103090008601109283010E94F2178BB1837E90917A
:1030A0008501892B8BB98BB18F7190918401892B0C
:1030B0008BB908958AB18C618AB9209A8AB1806EE1
:1030C0008AB9E1E8F0E080818F7E8083808188602A
:1030D0008083E0E8F0E080818C7F808380818F7046
:1030E0008083EEE6F0E08081887F808314BC15BC8D
:1030F0008081816080830895CF93DF93C0918101A7
:10310000D09182012097B9F081E0809355016091C0
:103110006B0170916C0180916D0190916E019B012A
:10312000AC010E949E36698B7A8B8B8B9C8B1092A4
:10313000820110928101DF91CF9108952F923F92E9
:103140004F925F926F927F928F929F92AF92BF92B7
:10315000CF92DF92EF92FF920F931F93CF93DF9363
:10316000CDB7DEB7E5970FB6F894DEBF0FBECDBF83
:1031700080912805807709F40AC220E030E0A90197
:1031800060916B0170916C0180916D0190916E0165
:103190000E9460348111FBC103C68091810190912E
:1031A0008201892B09F4FAC180918701F6E0F89F2A
:1031B000F0011124E455FE4FFE83ED83809154010C
:1031C000828320918101309182013E872D87D90130
:1031D0009596BC91BCA7F901F6A1FDA7D9019796D8
:1031E000BC91BEA7F901F0A5FFA720915E01309127
:1031F0005F0140916001509161016CA57DA58B2F0D
:103200009F2F0E94863368A779A78AA79BA720E0F3
:1032100030E0A9010E94603487FF04C018A619A6F7
:103220001AA61BA620917701288F30917801398F3B
:10323000409179014A8F50917A015B8F80916F01A3
:103240008C8F909170019D8FA0917101AE8FB09184
:103250007201BF8FE0917B01E8A3F0917C01F9A39B
:1032600020917D012AA330917E013BA3409167010B
:103270004CA3509168015DA3809169018EA3909148
:103280006A019FA3209173013091740140917501EF
:103290005091760128AB39AB4AAB5BAB30916B01F7
:1032A000398340916C01498720906D0130906E0107
:1032B000509166015F878CA58C8B9DA59D8BAEA5DB
:1032C000AE8BBFA5BF8B3EE3C32E33ECD32E3EE2C5
:1032D000E32E39E3F32E188A198A1A8A1B8A2601EB
:1032E0003701EF85E111B4C3AD85BE8591962D916F
:1032F0003D914D915C919497C701B6010E949E3615
:103300004B015C0120E030E040E05FE30E949E362C
:103310009B01AC0169817985C1010E9487339B01C2
:10332000AC01C701B6010E949E369B01AC016C89BD
:103330007D898E899F890E9486338B018DAB9CABE2
:10334000288D398D4A8D5B8D0E94603487FF86C33E
:10335000288D398D4A8D5B8D6CA57DA58EA59FA589
:103360000E9486339B01AC010E9487336B017C0174
:103370002C8D3D8D4E8D5F8D69817985C1010E94B7
:1033800087339B01AC01C701B6010E9467346B0112
:103390007C0128A139A14AA15BA1688D798D8A8D14
:1033A0009B8D0E946034882309F455C3B1E0BF8728
:1033B000FC8DF9832D8D29872E8C3F8C088D198DDE
:1033C0003A8D3DAB4B8D4CABA7019601688979894D
:1033D0008A899B890E948733688B798B8A8B9B8B28
:1033E000A30192010E94603487FDF2C328A539A58C
:1033F0004AA55BA5B8018DA99CA90E946336181641
:103400000CF4DCC389819985D10180936B01909381
:103410006C01A0936D01B0936E01FF85F09366017E
:1034200040905A0150905B0160905C0170905D018A
:1034300098014DA95CA9C301B2010E949E3669831F
:103440007A838B839C830E944D346B017C01609155
:1034500056017091570180915801909159010E9435
:103460004D344B015C01A70196010E9486330E94F6
:10347000D43469877A878B879C87E985FA85AD8103
:10348000BE81ED93FC93309709F4CDC32091620186
:103490003091630140916401509165016889798997
:1034A0008A899B890E9487332B013C0129813A81BB
:1034B0004B815C81C501B4010E9486339B01AC0144
:1034C000C301B2010E9467344B015C0129813A813A
:1034D0004B815C81C701B6010E948633A50194012E
:1034E0000E949E3660936201709363018093640131
:1034F0009093650120EC31EE44E65EE4C501B40131
:103500000E949E360E944D340E94D434603DB7E044
:103510007B078105910508F0ACC3ED81FE81158222
:10352000AD81BE8114967C936E9313978091860132
:10353000809387018F5F863009F4D4C3809386011E
:1035400020916701309168014091690150916A01B1
:10355000B8018DA99CA90E94633618160CF0C5C34A
:10356000E0918101F0918201C801ADA9BCA985A3B8
:1035700096A3A7A3B0A789819A81AB81BC818093D0
:10358000560190935701A0935801B093590190911F
:10359000880180918601981300CE02C40E94C02346
:1035A0001C019093820180938101009709F4F8C374
:1035B0008091550110912805882319F0109255012A
:1035C000BEC0809154018F5F853019F08093540103
:1035D00002C010925401E091540121E12E9FF001AC
:1035E0001124E053FE4FF0938001E0937F01D1015D
:1035F0008C91808311964D915D916D917C91149782
:1036000003E0440F551F661F771F0A95D1F74183CA
:1036100052836383748315964D915D916D917C9176
:10362000189783E0440F551F661F771F8A95D1F7BF
:10363000458356836783708719964D915D916D918F
:103640007C911C9793E0440F551F661F771F9A9536
:10365000D1F741875287638774871D966D917D915D
:103660008D919C9150976B017C0123E0CC0CDD1C6B
:10367000EE1CFF1C2A95D1F7C586D686E786F08A10
:103680000E94003560935601709357018093580152
:1036900090935901F10125A136A147A150A50E949F
:1036A00067349B01AC0160935A0170935B01809376
:1036B0005C0190935D0160E070E080EA9FE30E940E
:1036C000673460935E0170935F0180936001909313
:1036D00061011092620110926301109264011092D4
:1036E0006501812F8077E1F0609173017091740121
:1036F000809175019091760160936B0170936C01DC
:1037000080936D0190936E019B01AC010E949E36E7
:10371000D10151966D937D938D939C9354970FC0D7
:10372000F10161897289838994890E942B376093A2
:103730006B0170936C0180936D0190936E011092F8
:103740006701109268011092690110926A01D1011B
:1037500091968D909D90AD90BC909497A501940109
:1037600060E070E080E09FE30E9467342B013C0141
:103770001077F101C5A0D6A0E7A0F0A4112309F4A9
:103780004DC0F2E0F0936601D10151962D913D912B
:103790004D915C9154972D833E834F8358870E94AF
:1037A0009E369B01AC01C701B6010E9486332B01F6
:1037B0003C0120E030E0A9010E94603487FF1DC079
:1037C000A5019401C501B4010E948733A7019601A8
:1037D0000E949E369B01AC016D817E818F81988510
:1037E0000E9486330E942B3760937301709374019B
:1037F0008093750190937601D7CC409267015092E7
:1038000068016092690170926A01109273011092CE
:1038100074011092750110927601C6CC1092660167
:10382000C0927701D0927801E0927901F0927A010A
:103830000E94D0234B015C0160937301709374016B
:1038400080937501909376019B01AC010E949E3696
:1038500069837A838B839C8300918101109182011B
:10386000D80195962D913D914D915C91989729871E
:103870003A874B875C8751962D913D914D915C9194
:1038800054972D833E834F8358879B01AC016D81F4
:103890007E818F8198850E9486339B01AC01C30194
:1038A000B2010E949E369B01AC0169857A858B85A9
:1038B0009C850E94873320E030E040E05FE30E9477
:1038C0009E366B017C0120E030E0A9010E94633646
:1038D00018160CF0ACC029853A854B855C85C7016C
:1038E000B6010E94603487FF8EC0F801858C968CEB
:1038F000A78CB0A029813A814B815C81C501B401BC
:103900000E9486339B01AC01C301B2010E949E3626
:1039100060937B0170937C0180937D0190937E0185
:10392000A70196010E94603487FF3DC0C501B40124
:103930000E942B3760936F01709370018093710127
:1039400090937201A50194016D817E818F8198858C
:103950000E946034811104C0F1E0F093660124CC30
:103960002D813E814F815885C501B4010E94863367
:103970009B01AC01C301B2010E949E369B01AC01C8
:1039800060917701709178018091790190917A012D
:103990000E94863360937701709378018093790158
:1039A00090937A0101CCC0927701D0927801E09295
:1039B0007901F0927A01C0927B01D0927C01E09271
:1039C0007D01F0927E01D80191966D917D918D914E
:1039D0009C9194979B01AC010E948733A7019601AB
:1039E0000E949E3629813A814B815C810E948733F7
:1039F0000E942B3760936F01709370018093710167
:103A000090937201D1CBB2E0B093660180916B01CB
:103A100090916C01A0916D01B0916E0180936F0146
:103A200090937001A0937101B0937201BDCB10927D
:103A30007701109278011092790110927A018092A8
:103A40006F0190927001A0927101B0927201ACCBA3
:103A5000E13061F041C0E2E0EF87AACCA50194011A
:103A600069817985C1010E9487337CC0A7019601D5
:103A70006C8D7D8D8E8D9F8D0E949E369B01AC013D
:103A80006C897D898E899F890E9486338B018DABDD
:103A90009CAB28A139A14AA15BA10E94603487FF99
:103AA00093CC28A139A14AA15BA16C897D898E891B
:103AB0009F890E9486332C8D3D8D4E8D5F8D0E9497
:103AC00067346B017C0108A119A15AA15DAB8BA1E0
:103AD0008CAB92E09F8778CCAD85BE8591962D9179
:103AE0003D914D915C919497C701B6010E949E361D
:103AF0004B015C019B01AC0169817985C1010E9488
:103B0000633618169CF520E030E040E05FE3C50125
:103B1000B4010E949E369B01AC0169817985C10187
:103B20000E9486339B01AC01C701B6010E949E36FC
:103B30009B01AC016C897D898E899F890E948633A7
:103B40008B018DAB9CAB2CA13DA14EA15FA10E942E
:103B5000633618165CF4A501940169817985C10169
:103B60000E948633698379871C012ECC2CA13DA14C
:103B70004EA15FA16C897D898E899F890E948633C1
:103B80009B01AC010E9487336B017C0128A939A9F4
:103B90004AA95BA969817985C1010E9487339B018C
:103BA000AC01C701B6010E9467346B017C010CA116
:103BB0001DA1BEA1BDABEFA1ECAB06CC2EE333EC57
:103BC0004EE259E3C301B2010E9487332B013C014D
:103BD000288939894A895B89C301B2010E948633E9
:103BE0006B017C012CA13DA14EA15FA1B8018DA963
:103BF0009CA90E94633618167CF089819985D101B1
:103C000080936B0190936C01A0936D01B0936E0152
:103C10003F853093660104CC0C8B1D8B4DA94E8BD8
:103C20005CA95F8B5ECB80912805807709F42ECC50
:103C300010926B0110926C0110926D0110926E0146
:103C4000109262011092630110926401109265015A
:103C5000C0925601D0925701E0925801F09259015A
:103C6000A3019201C701B6010E946734AD85BE85EC
:103C700070C0603AFFE07F078105910510F4E1E034
:103C800009C06034FFE17F078105910510F4E2E08F
:103C900001C0E3E0AD81BE811596EC93AD81BE819C
:103CA00015962C911597022E04C0969587957795B9
:103CB00067950A94D2F7E985FA8502C0EE0FFF1FD7
:103CC0002A95E2F7ED93FC9361157105F1E08F07FA
:103CD000910508F425CC2FEF3FEFED81FE81348371
:103CE000238324CC109286012BCC20E030E0A90164
:103CF000B8018DA99CA90E94633618160CF049C022
:103D000010926B0110926C0110926D0110926E0175
:103D10001092620110926301109264011092650189
:103D2000C0925601D0925701E0925801F092590189
:103D3000009181011091820120915A0130915B0123
:103D400040915C0150915D01C701B6010E9467344A
:103D5000D80195966D937D938D939C939897E59656
:103D60000FB6F894DEBF0FBECDBFDF91CF911F918C
:103D70000F91FF90EF90DF90CF90BF90AF909F900A
:103D80008F907F906F905F904F903F902F900C940A
:103D9000252710928201109281010E94AC23F7CB5B
:103DA000E5960FB6F894DEBF0FBECDBFDF91CF9181
:103DB0001F910F91FF90EF90DF90CF90BF90AF9049
:103DC0009F908F907F906F905F904F903F902F903B
:103DD0000895F999FECF92BD81BD81E08FBB80B57A
:103DE0000895F894F999FECF92BD81BD81E08FBB13
:103DF00040B54627842F992787FD9095262F30E0E0
:103E000082239323892B39F06F3F19F060BD84E042
:103E100006C084E104C0442321F060BD84E28FBB6E
:103E2000F99A789408959F92AF92BF92CF92DF92C1
:103E3000EF92FF920F931F93CF93DF938C017A0140
:103E40006B01C40ED51EEB01912C5C01A61AB70ABA
:103E5000CE018A0D9B1DCC15DD0591F0911009C096
:103E6000692D772767FD7095272F221F2227221F94
:103E700001C021E06991922E960E0E94F11EE8CFBA
